:020000040000FA
:0600000060283F300130D2
:08000800A000030EA100831209
:100010008B1C2E288B1031181328B11C2E2864300D
:100020000102031C2D281428152816281728182823
:1000300019281A281B283110B114A810031005190B
:100040000314AA0DA90DA80DB00B2E2831152A08EE
:10005000AF002908AE002808AD00B11081010B11D6
:0A006000210E8300A00E200E0900FF
:1000C000203084008001840A80300402031C6228EE
:1000D0001230B000442283160C308505870183124C
:1000E000850187010730990000309A00103083168F
:1000F0008E008312603083168F00831200308316C7
:1001000091009F008312C830831681008312313022
:100110009000003083168C00831210308B003D1B42
:10012000BE013D1BBF013D1F6F2281018E018F016A
:100130000B118B100B108C018B17AD203119C320C4
:100140001622B30BAB28031085190314BA0DF03037
:100150003A020319752170229D28640031180800A5
:100160000B1D08000B11B11031141230B000051D29
:10017000BE2832148316011383120800321083162E
:10018000011783120800321CCA282D090339AD005B
:10019000AE09AF09E4302F02F0300319AF004C3044
:1001A0002F020C300319AF006C302F023C300319C2
:1001B000AF00EC302F02FC300319AF00B3302F0238
:1001C000F3300319AF001B302F020F300319AF00BB
:1001D0003B302F023F300319AF00BB302F02FF30FE
:1001E0000319AF0031110130B7008B1320303707EE
:1001F00083169B001C141A088312A400A500251066
:100200001030370783169B001C141A088312A300B2
:100210000030370783169B001C141A088312A200B3
:100220008B1722082D02031D6F2923082E06FC3987
:10023000031D6F29AF13AF12AF11AF1024082F02A7
:10024000031D462901303702031D2B293E182B2997
:100250003E14B117532202303702031D3429BE1851
:100260003429BE14B117562203303702031D3D292D
:100270003E193D293E15B117592204303702031D9E
:100280004629BE194629BE15B1175C2225082F0242
:10029000031D6F2901303702031D53293E1C5329CA
:1002A0003E10B1175F2202303702031D5C29BE1CCD
:1002B0005C29BE10B117632203303702031D652984
:1002C0003E1D65293E11B117672204303702031D18
:1002D0006E29BE1D6E29BE11B1176B226F29B70A98
:1002E0000530370203180800F528B601B30196302F
:1002F000B4000130B5000130B70085018701B113AA
:10030000E621AD20B30B9E29031085190314BA0D05
:10031000F0303A020319D629B41F8501B41F8701B2
:10032000B40B9E293708B6080319B60003199C2997
:10033000FF3085008700B6039630B400311D812957
:100340003111321CA8292D090339AD00AE09AF09BE
:1003500051302F0655390319BD2905302F0655395F
:100360000319BD2915302F0655390319BD295530FC
:100370002F0655390319BD298129AF13AF12AF11CB
:10038000AF108B1320303707BC002F08BB0024228E
:1003900010303707BC002E08BB002422003037077E
:1003A000BC002D08BB0024228B17E02185018701AA
:1003B000B70AB60105303702031C81296F220800F5
:1003C0000430370203190800850187016430B90041
:1003D00033300F1E85000F1A8501FF300F1A87007A
:1003E0000F1E8701AD20311DE8293111321CFD2976
:1003F0002D090339AD00AE09AF0951302F0655392B
:100400000319E62905302F0655390319E629153059
:100410002F0655390319E62955302F06553903198A
:10042000E629B90BE829850187010800B11F0800FA
:10043000B1131030BC003E08BB0024223030BC0099
:100440003F08BB00242208003C088B1383169B0046
:100450001C141A0883128B173B02031908008B1314
:100460003B0883161C159A0083123C0883169B00D8
:1004700055309D00AA309D009C1464009C183D2AB4
:100480001C1183128B170800831600309B001C146C
:100490001A088312BD00831610309B001C141A0822
:1004A0008312BE0008000130BE0008000230BE000A
:1004B00008000430BE0008000830BE0008008501B6
:1004C00087013E10080085018701BE1008008501E4
:1004D00087013E11080085018701BE110800080050
:1004E0008F08031908008F0103303E050319D82A2D
:1004F00002303E05031D51105408EB3C0318051251
:100500005118852AD40B902A8A2AD4035408C83C4F
:10051000031C902A0516F530D4005108013AD10089
:1005200002303E05031DD1105508E63C0318851224
:10053000D1189D2AD50BA82AA22AD5035508B93C63
:10054000031CA82A8516F030D5005108023AD100C4
:1005500002303E05031D51115608DC3C03180510FE
:100560005119B52AD60BC02ABA2AD6035608B63C6A
:10057000031CC02A0514E630D6005108043AD10005
:1005800002303E05031DD1115708F03C03188510B9
:10059000D119CD2AD70BD82AD22AD7035708D73C4E
:1005A000031CD82A8514FA30D7005108083AD10024
:1005B0000C303E050319282B3E1DE42A54083C3C10
:1005C000031CE42A85018701D40B0800D0034630C0
:1005D000D4000B305002031DEE2A05160A305002DB
:1005E000031DF32A851609305002031DF82A05144D
:1005F00008305002031DFD2A851407305002031DE8
:10060000022B871406305002031D072B07150530F7
:100610005002031D0C2B071404305002031D112B34
:10062000871603305002031D162B071602305002A6
:10063000031D1B2B871501305002031D1F2B123089
:100640005002031C0800850187010C30D00008000F
:1006500020303E050319482BD40B332B0508103AE4
:1006600085008230D400D50B3A2B0508203A85004E
:100670007D30D500D60B412B0508013A850073303B
:10068000D600D70B482B0508023A85008730D700E3
:0E06900040303E0503194E2B850187010800FE
:084000000600000006000200AA
:02400E00CC33B1
:10420000010003000300030003000200020002009B
:10421000020000000000FF00FF00FF00FF00FF00A1
:10422000000000000000000000000000000000008E
:104230000000C000C000FF00FF00FF00FF00FF0003
:104240000100510005001500550051000500150042
:10425000550051000500FF00FF00FF00FF00FF00B8
:104260000000FF00FF00FF00FF00FF00FF00FF0055
:10427000FF00FF00FF00FF00FF00FF00FF00FF0046
:10428000FF00FF00FF00FF00FF00FF00FF00FF0036
:10429000FF00FF00FF00FF00FF00FF00FF00FF0026
:1042A000FF00FF00FF00FF00FF00FF00FF00FF0016
:1042B000FF00FF00FF00FF00FF00FF00FF00FF0006
:1042C000FF00FF00FF00FF00FF00FF00FF00FF00F6
:1042D000FF00FF00FF00FF00FF00FF00FF00FF00E6
:1042E000FF00FF00FF00FF00FF00FF00FF00FF00D6
:1042F000FF00FF00FF00FF00FF00FF00FF00AA001B
:00000001FF
